:100000000C9462020C9400000C9400000C9400000C
:100010000C9400000C9400000C9400000C94000060
:100020000C9400000C94DA030C9400000C9411035F
:100030000C9400000C9400000C9400000C94000040
:100040000C9400000C9400000C9400000C94000030
:100050000C940000C1AEB6BAC1FFFFBD80BFFFFF68
:100060008DB6B6B6B9FFDDBEB6B6C9FFE7EBED801B
:10007000EFFFD8BABABAC6FFC3B5B6B6CFFFFE8E89
:10008000F6FAFCFFC9B6B6B6C9FFF9B6B6D6E1FFB7
:10009000F7F7F7F7F7FFC1BEBEBEC1FFF7F7F7F7F7
:1000A000F7FF80F6F6FEFEFFC1BEBEBEC1FF80FDBB
:1000B000FBF780FFFFFFFFFFFFFFBE80BEBEC1FF5B
:1000C00080F7F7F780FFFFFFFFFFFFFFFFBD80BF57
:1000D000FFFFD8BABABAC6FFB7ABABABDBFFC1BE46
:1000E000BEBEC1FF80F6F6FEFEFF80F6F6FEFEFF06
:1000F000FFFFFFFFFFFF80F6E6D6B9FFD9B6B6B621
:10010000CDFFFFFFFFFFFFFF80B6B6B6BEFF9CEB43
:10011000F7EB9CFFFFFFFFFFFFFFC1BEBEBEDDFF91
:10012000BE80BEBEC1FFFFFFFFFFFFFF80F7F7F7F6
:1001300080FFF7F7F7F7F7FFC1BEAEDEA1FF7C3E09
:10014000F97CF3F9E7F3CFE79FCF3F9F003EF97CBF
:10015000F3F9E7F3CFE79FCF3F9F7F3E007CF9F9AC
:10016000F3F3E7E7CFCF9F9F3F3F7F7EFFFCFFF991
:10017000FFF3FFE7FFCFFF9FFF3FFF3FFF9FFFCF53
:10018000FFE7FFF3FFF9FFFC7F7E3F3F9F9FCFCF4D
:10019000E7E7F3F3F9F9007C7F3E3F9F9FCFCFE77E
:1001A000E7F3F3F9F97C003E3F9F9FCFCFE7E7F3FA
:1001B000F3F9F97C7C3EFF3FFFCFFFF7FFF97F7E2D
:1001C0009F3FE71FFB0FFD07FE03FE03FD07FB0F2D
:1001D000E71F9FBF7F7EFFF9FFF7FFCFFF3FFF3F86
:1001E000FFCFFFF7FFF97F7E9F3FE71FFB0FFD0764
:1001F000FE03FE03FD07FB0FE71F9FBF7F7EFFF996
:10020000FFF7FFCFFF3FFF3FFFCFFFF7FFF97F7EF5
:100210009F3FE71FFB0FFD07FE03FE03FD07FB0FDC
:10022000E71F9FBF7F7EFFF9FFF7FFCFFF3FFFFF75
:100230009324FFFF4992FFFF9324FFFF4992FFFFA2
:100240009324FFFF4992FFFF9324FFFFFFFF9324B6
:10025000FFFF4992FFFF9324FFFF4992FFFF932482
:10026000FFFF4992FFFF9324FFFFFFFF9324FFFF4F
:100270004992FFFF9324FFFF4992FFFF9324FFFF62
:100280004992FFFF9324FFFFFFFF9324FFFF499252
:10029000FFFF9324FFFF4992FFFF9324FFFF499242
:1002A000FFFF9324FFFFFF3FFF1FFF0FFF07FF43E9
:1002B000FF61FF307F183F0C1F060F7F0700030010
:1002C00001000000FF3FFF1FFF0FFF07FF43FF611B
:1002D000FF307F183F0C1F060F7F0700030001004F
:1002E0000000FF3FFF1FFF0FFF07FF43FF61FF30CD
:1002F0007F183F0C1F060F7F07000300010000005E
:10030000FF3FFF1FFF0FFF07FF43FF61FF307F1815
:100310003F0C1F060F7F0700030001007FFE3FFC1C
:100320009FF9CFF367E6B3CDD99BEC37D99BB3CD1B
:1003300067E6CFF39FF93FFC7FFE7FFE3FFC9FF90E
:10034000CFF367E6B3CDD99BEC37D99BB3CD67E646
:10035000CFF39FF93FFC7FFE7FFE3FFC9FF9CFF379
:1003600067E6B3CDD99BEC37D99BB3CD67E6CFF326
:100370009FF93FFC7FFE7FFE3FFC9FF9CFF367E6CE
:10038000B3CDD99BEC37D99BB3CD67E6CFF39FF9BB
:100390003FFC7FFEFF7FFF1FFFC7FFF17F3C1FCFAA
:1003A000C7F3F37CC7F31FCF7F3CFFF1FFC7FF1FED
:1003B000FF7FFF7FFF1FFFC7FFF17F3C1FCFC7F30A
:1003C000F37CC7F31FCF7F3CFFF1FFC7FF1FFF7F09
:1003D000FF7FFF1FFFC7FFF17F3C1FCFC7F3F37CF9
:1003E000C7F31FCF7F3CFFF1FFC7FF1FFF7FFF7FDA
:1003F000FF1FFFC7FFF17F3C1FCFC7F3F37CC7F39D
:100400001FCF7F3CFFF1FFC7FF1FFF7F07E007E023
:100410007FFE07E007E0FFFF3FE03FE0BFE4BFE40F
:10042000FFFF07E007E0FFE7FFE7FFFF07E007E068
:10043000FFE7FFE7FFFF7FF03FE0BFEF3FE07FF028
:10044000FFFFFFFFFFFF010001003C0060025400BE
:1004500006009C0290001200A20296001200B40254
:10046000A8001200C602BA001200D802CC00180080
:10047000EA02DE0012000203F60012001403080173
:10048000120026031A01120038032C0178004A03D7
:100490003E017800C203B60178003A042E027500CE
:1004A000B204A60278002A051C037800A205940372
:1004B0003A001A060C0401005406460401000D001F
:1004C00048040000F894EE27ECBBF1E0FBBFEBBF63
:1004D000E5BFF8E1F1BDE1BD8DE0A2E0BB27ED9302
:1004E0008A95E9F780E098E0A0E6ED930197E9F7B7
:1004F000EAE4F4E085919591009761F0A591B591BA
:1005000005901590BF01F00105900D920197E1F75C
:10051000FB01F0CFEFE5EDBFE8E0EEBFC0E6D2E0D3
:100520000C94800EE4EA03C0E4E901C0E4E8E6BF0D
:10053000E2E0F0E00E945D100895E881E3B9F6DFA3
:1005400021960895F3DFE3B108951A931981A981E3
:100550000E946110A0E1EA02602DA12F0E946710A5
:10056000E62BE9830E946D10E981EA93E6DFDCDF88
:1005700018811DC01A930A930E946D10D3DFE1ED1C
:10058000EA93DBDFDFDF1E2FCFDF012F0E94771022
:10059000E0E1F0E00E94CC13AAE0EA02F001AE2F05
:1005A000E02FEF70EA0F1E2FE12F198108812396AB
:1005B00008951A9310E0183088F5ED81E07811F471
:1005C000C79801C0C79AEC81E07811F4C69801C0C1
:1005D000C69AEB81E07811F4C59801C0C59AEA810A
:1005E000E07811F4C49801C0C49AE981E07811F46C
:1005F000C39801C0C39AC29AC298ED81EE0FED83F1
:10060000EC81EE0FEC83EB81EE0FEB83EA81EE0FD2
:10061000EA83E981EE0FE9831F5FCDCF188126962B
:1006200008950A921A92FA926A937A938A939A9305
:10063000AA93BA93EA93FA93EFB7EA93E0E0E2BFA2
:100640005394ECE0E51531F45524E0913808EF5F60
:10065000E0933808A0913808A53018F0E0E0E09366
:100660003808E0913808E03011F00C947703E0E0AE
:10067000E2BBEBBB0E947A10E450F84FE081EA93B2
:10068000FD01E85FF74FE081EA93F001EC5EF74F80
:10069000E081EA93FB01E05EF74FE081EA93FB0122
:1006A000E45DF74F0E9480100E947A10E054F84FEA
:1006B000E081EA93FD01E453F84FE081EA93F00111
:1006C000E852F84FE081EA93FB01EC51F84FE081EA
:1006D000EA93FB01E051F84F0E948010C198C19A43
:1006E000E5E0E9BFE0E0FAEFFDBDECBD39C00E94F6
:1006F0007A10EC56F94FE081EA93FD01E056F94F8C
:10070000E081EA93F001E455F94FE081EA93FB01BF
:10071000E854F94FE081EA93FB01EC53F94F0E9452
:1007200080100E947A10EA5AF94FE081EA93FD01A5
:10073000EE59F94FE081EA93F001E259F94FE08177
:10074000EA93FB01E658F94FE081EA93FB01EA578F
:10075000F94F0E948010E0E0E2BBEBBBC198C19A68
:10076000E8E05E1630F4E52DA1E00E949B13E2BBA9
:1007700007C0E52DF0E03897A1E00E949B13EBBB8A
:100780000E94841019F4E1E0ED1509F005C0A1E024
:10079000B0E0E1E00E94F913E991EFBFF991E9912E
:1007A000B991A9919991899179916991F99019904B
:1007B00009901895EA93EFB7EA93E0913808E03092
:1007C00019F4E0E0E2BBEBBBE1E0E9BFE991EFBF88
:1007D000E99118951A930A9310E01031B8F40E9429
:1007E000891000E00C3380F40E948C100E948F105E
:1007F000EC56F94F0E9494100E9499100E949F108D
:100800000E94A3100F5FEECF1F5FE7CF18C01A93AF
:100810000A9310E0103198F40E94891000E00C3324
:1008200060F40E948C100E94B010EA5AF94F0E94A6
:10083000B5100E94BD100F5FF2CF1F5FEBCF099183
:10084000199108951A930A930E94D21011F40C94EE
:100850006F040E94D71009F442C010E01C3340F42A
:100860000E94DD100E94E0100E94EE101F5FF6CF84
:1008700010E0103198F50E9489101830B8F400E0AB
:100880000C3398F40E94FD100E940111E45FF84FB0
:100890000E9409110E94BD100E948C10A45FB84FE5
:1008A000EC91EE0FEC930F5FEBCF16C000E00C3332
:1008B00098F40E94FD100E940111E053F94F0E942C
:1008C00009110E94BD100E948C10A053B94FEC91E9
:1008D000EE0FEC930F5FEBCF1F5FCBCFB5CFECC12B
:1008E0001A930A930E94D21011F40C94BB040E9434
:1008F000D71009F440C010E01C3340F40E94DD1012
:100900000E94E0100E94EE101F5FF6CF10E0103141
:1009100088F50E9489101830B0F400E00C3390F490
:100920000E94FD100E9415110E9419110E94FD10D5
:100930000E949F100E94A3100E948C100E942611FA
:100940000F5FECCF15C000E00C3390F40E94FD1057
:100950000E9415110E942E110E94FD100E949F10EE
:100960000E94A3100E948C100E943B110F5FECCFDD
:100970001F5FCDCFB7CFA0C11A930A9310E01C33ED
:1009800040F40E94DD100E94E0100E94EE101F5FF4
:10099000F6CF0E94D21061F10E94D71049F110E009
:1009A0001C3328F50E94DD10E053F94FE081E093FD
:1009B00091060E94DD10E45FF84FE081E093CF06DE
:1009C00000E00B3380F40E948C100E94B0100E9453
:1009D00043110E948C100E948F10EB56F94FE0815A
:1009E000EC930F5FEECF0E9489101F5FD9CFD1CF5C
:1009F00063C11A930A9310E01C3340F40E94DD1087
:100A00000E94E0100E94EE101F5FF6CF0E94D210ED
:100A100081F10E94D71069F11BE3113048F10E9467
:100A2000DD10E053F94FE081E09356060E94DD109F
:100A3000E45FF84FE081E09394060BE30130A0F00F
:100A40000E948C100E94B0103197EA5AF94FE08151
:100A5000EC930E948C100E948F103197EC56F94F46
:100A6000E081EC930150EACF0E9489101150D5CF5C
:100A7000CDCF22C11A9310E01F3300F50E94DD1084
:100A8000DF01E053F94FBF01FD01E85BF84F0F01B3
:100A90000E9477100E9448110E944F11DF01E45F0D
:100AA000F84FBF01FD01EC57F84F0F010E9477107E
:100AB0000E945211DB01EC931F5FDECF2CC01A9312
:100AC00010E01C3340F40E94DD10E053F94FAEEF0C
:100AD000A0831F5FF6CFE8EFE093D006ECEFE09342
:100AE000D506E093DA06E8EFE093DF06ECEFE0935B
:100AF000E406E093E906E8EFE093EE06ECEFE0931E
:100B0000F306E093F806E8EFE093FD06ECEFE093E0
:100B10000207E0930707199108951A930A9300E0DA
:100B20000C3378F40E945911E45FF84F0F010E94D2
:100B30008C10A053B94FEFEFEC93D001EC930F5F03
:100B4000EFCFBDDF0E945C110E9475110E945C1105
:100B50000E947B11E7760E9480110E9493110E94EF
:100B600075110E949B110E9493110E947B11E373E7
:100B70000E9480110E94AD110E94B5110E94801147
:100B80000E94AD110E947B11E0780E9480110E94AA
:100B9000BB110E9475110E949B110E94BB110E9403
:100BA0007B11E3730E9480110E94C3110E94751192
:100BB0000E949B110E94C3110E947B11E7760E9444
:100BC000CB110E94B5110E94CB110E947B11EE70D7
:100BD0000E94D511E053F94FDF01EC91EF700E94B4
:100BE000D5110E947B11E0780E94DF110E94B5119F
:100BF0000E94DF110E947B11EE70EC93AA81B0E09D
:100C0000A053B94FEC91E770EC93AA81B0E0A45FD8
:100C1000B84FEC91E0700E94E9110E94ED110E9422
:100C200075110E94F4110E94ED110E947B11EF7C5E
:100C30000E94E9110E94F7110E9475110E94F4119F
:100C40000E94F7110E947B11EF790E94E9110E9426
:100C5000FE110E9475110E94F4110E94FE110E9463
:100C60007B11EF730E94E9110E9405120E94751119
:100C70000E94F4110E9405120E947B11EF790E94DC
:100C8000E9110E940C120E9475110E94F4110E9439
:100C90000C120E947B11EF7CEC9310E01C3360F48B
:100CA0000E9477100E9413120E9416120E941B12BB
:100CB0000E941E121F5FF2CF1981088125960895A8
:100CC0001A93E0913908EF5FE0933908A091390851
:100CD000A43618F0E0E0E0933908A0913908AC336D
:100CE00030F4E09139080E942312E08101C0EFEF57
:100CF000E093650610E0103140F40E9477100E94E6
:100D000013120E9443111F5FF6CFE0915606E09345
:100D100093061DE21D3340F40E9477100E941312C7
:100D20000E9443111F5FF6CF21C31A930A9310E06C
:100D3000163088F50E94DD10E35FF84FBF01AA81ED
:100D40000E9461100E9427120E944F11ED5EF84F21
:100D5000BF01AA810E9467100E942712DB01EC9359
:100D6000EBEDE09347070E94DD10E55CF84FBF0113
:100D7000AB810E9461100E9427120E944F11EF5B0D
:100D8000F84FBF01AB810E9467100E942712DB0160
:100D9000EC931F5FCDCF00E00C3340F40E948C1029
:100DA0000E948F100E941E120F5FF6CF19810881DA
:100DB000249608951A9314E11A32A0F40E94DD10CB
:100DC000E053F94F0F010E9477100E9448110E94D2
:100DD000DD10E45FF84F0F010E9477100E9452115E
:100DE0001F5FEACFC3C21A93E5DF0E943312EB51B3
:100DF000F94FA9EFA0830E943312EA51F94FA0EFF7
:100E0000A0830E943312E951F94F0E943612E85133
:100E1000F94F0E943612E751F94FA0EFA0830E94CC
:100E20003312E651F94FA9EFA0830E943312EF5D10
:100E3000F84F0E943912EE5DF84F0E943912ED5DB5
:100E4000F84F0E943612EC5DF84F0E943612EB5DAF
:100E5000F84F0E943912EA5DF84FAFEFA08316E118
:100E60001A3260F40E9477100E9413120E94161228
:100E70000E941B120E941E121F5FF2CF1881229641
:100E800008952197E0E0E8830E940A1400E030E032
:100E900050E040E03F5F3C3308F030E0E2E0E39FA9
:100EA000F001EE55FA4FE081E093FB07E2E0E39FAB
:100EB000F001ED55FA4FE081E093370820E02B3345
:100EC000B0F4A22FB0E0A054B84F0E943C12EF53F0
:100ED000F84FE081EC93A22FB0E0A450B84F0E94ED
:100EE0003C12E350F84FE081EC932F5FE8CF4A9239
:100EF0007A921BDF403009F45F5F5C3008F041E01C
:100F0000413009F45150503009F440E0EEE1F0E096
:100F10000E945D105A9367DFEE81EF5FEE83AE8132
:100F2000A33010F40C942D08E0E0EE83C9DE0E949B
:100F3000D71011F44FDC92C0C3940E943F1219F4F1
:100F4000E8E7CE1608F403C0CC2444DC87C00E9436
:100F500045127016D9F0072D0E944B12E4E0EA9377
:100F600009DB8E2EE5E0EA9305DBBE2EE6E0EA9390
:100F700001DBAE2E0E9451124E1619F4E2E0E71585
:100F800008F404C0E0E0E093540668C010E01630B6
:100F900010F00C942D080E94DD10E85BF84FBF01A3
:100FA000A82D0E9461100E9427120E944F11E25B3F
:100FB000F84FBF01A82D0E9467100E9427120E94BF
:100FC0004F110F01EC5AF84F0E945612E65AF84F93
:100FD000BF01AB2D0E9461100E9427120E944F1189
:100FE000E05AF84FBF01AB2D0E9467100E942712F4
:100FF0000E944F110F01EA59F84F0E945612E4590E
:10100000F84F0F01ACE6B2E0EE27A10FBE1FEC9146
:10101000D001EC930E94DD100F01EE58F84FDF0174
:10102000F001E05AFD4FE081EC930E94DD10E8589A
:10103000F84FBF01AA2D0E9461100E9427120E9442
:101040004F11E258F84FBF01AA2D0E9467100E946D
:101050002712DB01EC931F5F9ACF1CCF0E94111463
:10106000279608951A9310E0163010F00C94780823
:101070000E94DD10E45CF84FBF01A42D0E946110B6
:101080000E9427120E944F11EE5BF84FBF01A42D62
:101090000E9467100E9427120E944F11E45FF84FD0
:1010A000BF01A72D0E9461100E9427120E944F11BC
:1010B000EE5EF84FBF01A72D0E9467100E94271215
:1010C0000E944F11E85EF84FBF01A62D0E946110EB
:1010D0000E9427120E944F11E25EF84FBF01A62D19
:1010E0000E9467100E942712DB01EC931F5FBCCFA8
:1010F0003DC11A9310E0163010F00C94BF080E9406
:10110000DD10E45CF84FBF01A82D0E9461100E9421
:1011100027120E944F11EE5BF84FBF01A82D0E94CD
:1011200067100E9427120E944F11E45FF84FBF0121
:10113000AB2D0E9461100E9427120E944F11EE5E9B
:10114000F84FBF01AB2D0E9467100E9427120E942A
:101150004F11E85EF84FBF01AA2D0E9461100E9456
:1011600027120E944F11E25EF84FBF01AA2D0E9484
:1011700067100E942712DB01EC931F5FBCCFF6C003
:10118000E8E14E1608F04424E1E04E1610F4E7E1E1
:101190004E2EECE37E1608F07724E1E07E1610F484
:1011A000EBE37E2EECE36E1608F06624E1E06E16AB
:1011B00010F4EBE36E2EE0E28E1610F0E1E08E2EDE
:1011C000E1E08E1610F4EFE18E2EEDE0BE1610F089
:1011D000E1E0BE2EE1E0BE1610F4ECE0BE2EE8E247
:1011E000AE1610F0E0E1AE2EEFE0EA1510F0E7E207
:1011F000AE2E08951A930A9311E03CDCCE9903C0F9
:101200001F5FCE9BFECF1830F9F411E0E3DAE0E087
:10121000EA936A929AD9E1E0EA937A9296D9E2E067
:10122000EA934A9292D9E3E0EA939A928ED9E4E063
:10123000EA938A928AD9E5E0EA93BA9286D9E6E0FF
:10124000EA93AA9282D95CC0143011F41F5FC2DA0B
:10125000113011F0153019F4E0E0E0938C061230F3
:1012600011F0163031F4EFEFE0938C06E0E0E093FC
:101270005D06133011F0173031F4E0E0E0936906B9
:10128000EFEFE0935D06113031F4CC9B4A94CD9B97
:1012900043940E945D12123031F4CC9B7A94CD9B22
:1012A00073940E945D12133031F4CC9B6A94CD9BF1
:1012B00063940E945D12153031F4CC9B8A94CD9BCF
:1012C00083940E946112163031F4CC9BBA94CD9B6A
:1012D000B3940E946112173031F4CC9BAA94CD9B39
:1012E000A3940E946112E4E6F0E0E7D600E00C333C
:1012F00030F412D714D70E941E120F5FF8CF7ECFA2
:10130000C9C01A9310E0163088F557D7E45CF84F3F
:101310000E9465120E94CC130E9427120E944F1156
:10132000EE5BF84F0E9465120E94D1130E942712B3
:101330000E944F11E85EF84FBF010E9451120E94B7
:101340006F120E94CC130E9427120E944F11E25E7E
:10135000F84FBF010E9451120E946F120E94D113D8
:101360000E942712DB01EC931F5FCDCF19910895E6
:101370001A930A9300E07EDBCE9903C0CE9BFECF8A
:101380000F5F023018F000E025DA84C0A0E0CC99AD
:10139000A1E0A03011F4003009F011C00E947412D5
:1013A000EF5F0E94F913E1500E947412E83128F0B7
:1013B000A4E0B0E0E0E00E94F913CC9BFECFA0E0F7
:1013C000CD99A1E0A03011F4003009F011C00E94C5
:1013D0007412E1500E94F913EF5F0E947412E13021
:1013E00028F4A4E0B0E0E7E10E94F913CD9BFECF22
:1013F000A0E0CC99A1E0A03011F4013009F011C0B7
:101400000E945112EF5F0E94F913E1500E945112A5
:10141000E83128F0A5E0B0E0E0E00E94F913CC9BB1
:10142000FECFA0E0CD99A1E0A03011F4013009F089
:1014300011C00E945112E1500E94F913EF5F0E9407
:101440005112E13028F4A5E0B0E0E7E10E94F91381
:10145000CD9BFECF56DF003019F4E0E0E0930607A5
:10146000013031F4EFEFE0930607E0E0E093E206AD
:10147000E4E6F0E022D610E01C3358F438D60E949F
:1014800013120E9416120E941B120E941E121F5F4E
:10149000F3CF72CF0991199108950E9479120E9499
:1014A0007E120E94851283D609F47AC00E947912B6
:1014B0000E947E120E947E120E948B1278D609F43E
:1014C0006FC088D90E9479120E948B120E948F12DD
:1014D000E5E0EA9305DA0E94961209F461C0E2EBB6
:1014E000F4E00E949912E2EBF4E00E949C1244DACC
:1014F0008ED90E94A112E3E0EA93A4D988D90E9470
:101500008F120E948B120E94961209F449C00E9409
:101510008F120E948512E2EAF5E00E9499120E9461
:10152000A6122ADAE2EAF5E00E949C1262DA6FD98A
:101530003ED6B1F1EAE3F4E00E9499124BD9EAE217
:10154000F5E00E949912EAE2F5E00E949C1251DA5D
:101550002ED631F1EAE3F4E00E949912EAE2F5E0D6
:101560000E949C12BDD936D9E2ECF3E00E94991298
:101570000E949612A9F0E2ECF3E00E949912E2ECCC
:10158000F3E00E94AD1235DAE2ECF3E00E94B21211
:10159000F3D90E94961221F00E943F1209F07DCFEC
:1015A00008950E940C1410E030E089DAE0E0EA933C
:1015B0000E94BA026E2E0E9445120E944B120E9497
:1015C00051124E1619F4E0E0E71509F004C0E0E00E
:1015D000E093540687C1EF81E03049F51F5F1C336B
:1015E00010F010E03F5FE2E0E19FF0010E94B712CF
:1015F000E093FB07E2E0E19FF00131960E94B71211
:10160000E093370800E00B3390F486D5A054B84F30
:1016100050D6EF53F84FE081EC937ED5A450B84FED
:1016200048D6E350F84FE081EC930F5FECCFAF81E9
:10163000A13099F41F5F103110F010E03F5F00E01F
:101640000C3358F469D5A054B84F33D6E054F84F52
:101650008CD50E94BD120F5FF3CFAF81A230B1F4E1
:101660001F5F103110F010E03F5F00E00C3370F4AA
:1016700053D5A450B84F1DD6E450F84F55D559D581
:101680000E94D2120E94D6120F5FF0CFAF81A43019
:1016900011F00C94900B1030B9F420E02C33A0F42E
:1016A000E22FD1D60E94E3120E94B712DB01EC9325
:1016B000E3D6EC57F84F0E94E31231960E94B7121E
:1016C000DB01EC932F5FEACF1F5F103110F010E0C9
:1016D0003F5F183098F400E00C3378F48ED50E9408
:1016E000E812EC57F84F95D548D716D5AC57B84FF8
:1016F000EC91EE0FEC930F5FEFCF12C000E00C33D4
:1017000078F47BD50E94E812E85BF84F82D535D794
:1017100003D5A85BB84FEC91EE0FEC930F5FEFCFC2
:10172000AF81A33011F00C94DC0B103099F420E061
:101730002C3380F4E22F87D646D719D7DB01EC9300
:101740009BD6EC57F84F3FD7319611D7DB01EC937E
:101750002F5FEECF1F5F103110F010E03F5F1830A9
:10176000B0F400E00C3390F448D5E450F84F0F018A
:10177000DBD4AE2FFB01E85BF84F32D713D716D777
:10178000CBD4A85BB84F35D70F5FECCF15C000E0C6
:101790000C3390F432D5E450F84F0F01C5D4AE2F7E
:1017A000FB01EC57F84F1CD7FDD600D7B5D4AC578A
:1017B000B84F1FD70F5FECCFEC813E1708F092C0F7
:1017C000E0913A08E61511F40C945C0C60923A082A
:1017D0004A927A926A92A1D9E0E0E41511F40C944D
:1017E0003E0CE1E0E41511F40C943E0CE2E0E4154B
:1017F00011F40C943E0CE3E0E41511F40C943E0C4F
:10180000E4E0E415D9F1E5E0E415C1F1E6E0E41522
:10181000A9F1E7E0E41591F1E8E0E41579F1E9E0F8
:10182000E41561F1EAE0E41549F1EBE0E41531F18A
:10183000ECE0E41519F1EDE0E41501F1EEE0E4155A
:10184000E9F0EFE0E415D1F0E0E1E415B9F0E1E111
:10185000E415A1F0E2E1E41589F0E3E1E41571F0AB
:10186000E4E1E41559F0E5E1E41541F0E6E1E415C1
:1018700029F0E7E1E41511F0E0E001C0E1E00E2E0F
:10188000A62DE0E00E94AC13E02111F0DF9A01C028
:10189000DF98F5D529F4E0915506EF5FE093550602
:1018A000A0915506AC3340F0E0E0E0935506E0939C
:1018B0003C080E94070416C07AD431F4E0E0E093BB
:1018C0003C080E94EA030EC0ECD54E1619F4E2E083
:1018D000E71508F406C0E0E0E0935406E0933C0806
:1018E00001C064CE0E941314289608951A9312E042
:1018F000CC9905C011500E94EA03CC9BFECFCD9934
:1019000005C01F5F0E94EA03CD9BFECF143009F48F
:1019100011E0103009F413E0113099F4E5E3E0939D
:101920003B08A0913B08AC3360F469D6F597EC54C2
:10193000FD4F6ED674D6EC54FD4FE081EC9376D615
:10194000F0CF123099F4E4E3E0933B08A0913B0818
:10195000AC3360F454D6F497E651FD4F59D66CD6AB
:10196000E651FD4FE081EC9361D6F0CF133099F44E
:10197000E4E3E0933B08A0913B08AC3360F43FD62E
:10198000F497E852FD4F44D657D6E852FD4FE08118
:10199000EC934CD6F0CFB8D311F4113009F00AC053
:1019A000CE9BFECFA0E0B0E0E1E04DD6A2E0B0E0FB
:1019B00052D61FC0A9D311F4123009F009C0CE9B32
:1019C000FECFA0E0B0E0E0E03ED60E94EA0311C006
:1019D0009BD311F4133009F00BC0CE9BFECFA3E0D4
:1019E000B0E0E1E00E94F913A0E0B0E034D601C01D
:1019F0007FCF81C11A9311E00E94EA03CC9905C000
:101A000011500E94EA03CC9BFECFCD9905C01F5F09
:101A10000E94EA03CD9BFECF143009F411E0103090
:101A200009F413E0113089F4E7E3E0933B08A09157
:101A30003B08AC3350F414D6A6E6B2E0A60FB71FAD
:101A4000EC91D001EC93F2D5F2CF123089F4E7E3B8
:101A5000E0933B08A0913B08AC3350F401D6ACE6D0
:101A6000B2E0A60FB71FEC91D001EC93DFD5F2CF17
:101A70001330C1F4E5E3E0933B08A0913B08AC339D
:101A800088F4F7D5EC56F94F0F01A6E6B2E0F6D58B
:101A9000F0D5F597EC56F94F0F01ACE6B2E0EED574
:101AA000C5D5EBCF113011F42FD309F007C0A2E058
:101AB000B0E0E1E0EBD5CE9BFECF19C0123011F4BF
:101AC00023D309F007C0A2E0B0E0E2E0DFD5CE9B6F
:101AD000FECF0DC0133011F417D309F007C0A2E0F8
:101AE000B0E0E3E0D3D5CE9BFECF01C087CF03C1EA
:101AF0001A9313E00E94EA03CE9BFECFCC9905C057
:101B000011500E94EA03CC9BFECFCD9905C01F5F08
:101B10000E94EA03CD9BFECF173009F411E010308C
:101B200009F416E0113099F4E5E3E0933B08A09145
:101B30003B08AC3360F463D5F597EE5FFC4F68D596
:101B40006ED5EE5FFC4FE081EC9370D5F0CF123094
:101B500099F4E5E3E0933B08A0913B08AC3360F4D3
:101B60004ED5F597EA5DFC4F53D559D5EA5DFC4F4C
:101B7000E081EC935BD5F0CF133099F4E4E3E0938C
:101B80003B08A0913B08AC3360F439D5F497E85C8E
:101B9000FC4F3ED57FD5E85CFC4FE081EC9346D509
:101BA000F0CF143099F4E5E3E0933B08A0913B08B3
:101BB000AC3360F424D5F597EC5EFC4F29D52FD5D6
:101BC000EC5EFC4FE081EC9331D5F0CF153099F409
:101BD000E5E3E0933B08A0913B08AC3360F40FD5FC
:101BE000F597EA53FD4F14D51AD5EA53FD4FE0811E
:101BF000EC931CD5F0CF163099F4E4E3E0933B0866
:101C0000A0913B08AC3360F4FAD4F497EE55FD4F45
:101C1000FFD440D5EE55FD4FE081EC9307D5F0CFD2
:101C2000163011F471D209F007C0CE9BFECF0E948E
:101C3000EA039EDB0E943A05153011F465D209F0E3
:101C400003C0CE9BFECFD6DE143011F45DD209F076
:101C500008C0CE9BFECFA1E0B0E0FDD4E1E0DE2ED7
:101C60004AC0123011F450D209F007C0CE9BFECF0B
:101C70000E94EA03BFDA0E943A05133011F444D2FD
:101C800009F005C0CE9BFECF0E94EA032FDE113083
:101C900011F43AD209F02EC00E94EA03CE9BFECF87
:101CA000E0E0EA93EA930E94A502E1E0EA93EEE124
:101CB000EA930E94A502E2E0EA93ECE0EA930E9434
:101CC000A502E3E0EA93E2E0EA930E94A502E4E0E1
:101CD000EA93E1E0EA930E94A502E5E0EA93ECE0F2
:101CE000EA930E94A502E6E0EA93E0E1EA930E940B
:101CF000A50201C003CF19910895CDD3C6D308958D
:101D0000A29AE5E0E9BFEAE0E2BFE2E0E3BFECED82
:101D1000FFEFFDBDECBDE1E0EEBD7894EFEFE4BB7D
:101D2000E7BBEFE0EABBEFEFE1BB0E943A05E0E082
:101D3000E0933E08A0913E08AC3340F4B2D4B5D451
:101D4000E450F84FAFEFA083B5D4F4CFE7E4E0B9A7
:101D5000EDE2E0933E08A0913E08AA3310F5A1D42D
:101D60000F01EE52F94FDF01F001BD97A9D40F0129
:101D7000E25FF84FDF01F001BD97A9D492D40F01C3
:101D8000BB97E053F94FDF01F0017E9799D40F0123
:101D9000BB97E45FF84FDF01F0017E9798D48AD4B7
:101DA000DACFE0E0E0933E08A0913E08A031C0F514
:101DB000EEE1F0E082D1A0913E08A830C0F4E0E06E
:101DC000E0933F08A0913F08AC3380F487D42DD234
:101DD00030D284D4B4D1B7D1A0913F08B0E036D28C
:101DE000E0913F08EF5FE0933F08ECCF17C0E0E0E1
:101DF000E0933F08A0913F08AC3380F46FD415D234
:101E00002DD26CD49CD19FD1A0913F08B0E033D2A9
:101E1000E0913F08EF5FE0933F08ECCF4BD4C4CF95
:101E2000E0EDF7E04AD10E94070467DFE8ECF0E05C
:101E300044D15AD34E1619F4E2E0E71508F403C072
:101E4000E1E0E09354062DD34E1619F4E2E0E715D5
:101E500008F403C0E0E0E0935406A0915406A130DA
:101E600021F4E1E0E9BFC09A05C0E0E0E9BFEBBBC7
:101E7000E2BBC098CE9906C0CE9BFECFE1E0E093D6
:101E80005406E9BF94D121F4A0915406A13009F081
:101E900011C0DD24E0E0E0933E08A0913E08AC33A1
:101EA00040F4FFD302D4E450F84FAFEFA08302D444
:101EB000F4CF1EDEA2E0B0E00E94ED13E13011F09D
:101EC000DED231F410D421F4A0915406A13009F0EF
:101ED000CBC00E94EA030E943A050E945F05E42DF0
:101EE00008D4E72DF0E0E053F94FAFE0A083E72DF1
:101EF00000D4E62DF0E0E053F94FA3E0A083E62DF7
:101F0000F8D3E0E0E0933D08A0913D08AC3328F51C
:101F1000EAE0F0E0D2D0E0913D08F0E0BF01DF015F
:101F2000EA5AF94F0F01FD01E053F94FA081FB017F
:101F3000E85BF84FE081EA23D001EC93A0913D08E3
:101F4000B0E0AC56B94FE0913D08F0E077D2E091B7
:101F50003D08EF5FE0933D08D7CFE1E0E0933C0818
:101F6000A0913C08A13031F4E3E0EA93C2D2E2E070
:101F7000EA9317DBA0913C08A13031F4E4E0EA9346
:101F8000B8D2E3E0EA930DDBA0913C08A13031F434
:101F9000E3E0EA93AED2E2E0EA9303DBA0913C08EF
:101FA000A13011F4ACD3FDDAA0913C08A13011F4BA
:101FB000A9D3F7DAA0913C08A13011F4A0D3F1DA4B
:101FC000A0913C08A13011F49DD3EBDAA0913C081C
:101FD000A13019F4E4E09BD3E4DAA0913C08A130ED
:101FE00019F4E3E094D3DDDAA0913C08A13011F4B8
:101FF00086D3D7DAA0913C08A13021F4E3E0EA933C
:10200000A5D2CFDAA0913C08A13049F4E0E0EA93F0
:10201000E2EAF5E0FA93EA93E5E0EA93C2DAA09106
:102020003C08A13031F4E4E0EA938BD2E1E0EA939A
:10203000B8DAA0913C08A13031F4E0E0EA9381D213
:10204000E5E0EA93AEDAA0913C08A13019F4E1E0B2
:102050005ED3A7DA14D231F0AAD021F0A0915406B1
:10206000A03009F401C079CFA0E0B0E00E94ED13E8
:10207000E13011F004D231F436D321F4A0915406AA
:10208000A13009F005C009DA0E94EA030E943A056E
:10209000F6D131F0A2E0B0E00E94ED13E23031F46D
:1020A00022D321F4A0915406A13009F004C00E946B
:1020B0003A050E944107B9CEFFCFFA93EA930C94F8
:1020C0008B13B0E0EAE0F0E00E94CC130895BB2748
:1020D000EAE0F0E00E94D11308950E949202E0ED40
:1020E000EA930E949D02EA81EA930C949D02A12F3B
:1020F000B0E00895E52DF0E0BF010F01DF01089584
:10210000E081EA930C94D902A0E0CE99A1E0A0303E
:102110000895E8E2F0E0D1CFA02FB0E00895AC56EA
:10212000B94FE02FF0E00895E081F0E0F595E795F4
:102130000895E068EC93E02FF0E0BF010895EA5ABB
:10214000F94F0F01F1CFAE2FFB01EC56F94FE081B3
:10215000E170E795E0E0E795EA2BD001EC93089574
:10216000AA5AB94FE02FF0E00895E081EE0FE16048
:10217000EC93E02FF0E0BF010895EC56F94F0F010A
:10218000E081EE0FAE2FFB01EA5AF94FE081F0E05B
:10219000E078F0700E94A5130E94A313EA2BD001EF
:1021A000EC930895EA81E150EA83EF5F0895A1E09E
:1021B000B0E00E94ED13E1300895E12FF0E00895C2
:1021C000E053F94FBF01E2E0E19FF001AB81BC8138
:1021D000AE0FBF1FEC91DB01EC93EFCFE45FF84F44
:1021E000BF01E2E0E19FF0013196AB81BC81AE0F0F
:1021F000BF1FEC91DB01EC930895E02FF0E0BF01ED
:102200000895EA5AF94F0F01E081EE0FAE2FFB015E
:102210000895E081F0E0E078F0700E94A5130E943C
:10222000A313EA2BD001EC93E8CFEC56F94F0F0142
:102230007BCFAE2FFB01E053F94FE081E170E795D2
:10224000E0E0E795EA2BD001EC930895A053B94F55
:10225000EC91F0E0F595E795EC930895AE2FFB0136
:10226000E45FF84FE081E170E795E0E0E795EA2B65
:10227000D001EC930895A45FB84FEC91F0E0F59590
:10228000E795EC930895E95AF94FE081EC930895AE
:10229000AA5AB94FEFEFEC93D001EC930895DB010C
:1022A000EC938BCFAC56B94FEFEFEC93D001EC939E
:1022B0000895E02FF0E00895AC81E5E0EA9FF00199
:1022C000DF01ECE3F0E00E94D113BF01AB81B0E08D
:1022D000ECE0F0E00E94CC13DB01AE0FBF1FDA96FA
:1022E000ECE3F0E00E94D1130895E053F94FDF01D1
:1022F000EC91EC930895E45FF84FDF01EC910895C1
:10230000EC93AC81E5E0EA9FF001DF01ECE3F0E063
:102310000E94D113BF01AB81B0E0ECE0F0E00E947D
:10232000CC13DB010895AE0FBF1FDB96ECE3F0E0AA
:102330000E94D1130895AC81E5E0EA9FF001DF012E
:10234000ECE3F0E00E94D113BF01AB81B0E0ECE020
:10235000F0E00E94CC13DB010895AE0FBF1FDC96A6
:10236000ECE3F0E00E94D1130895E053F94FDF0150
:10237000EC91EF770895AE0FBF1FDD96ECE3F0E030
:102380000E94D1130895AE0FBF1FDE96ECE3F0E07C
:102390000E94D1130895EC93EB81F0E0FB96DF01EE
:1023A000ECE3F0E00E94D1130895EC93EB81F0E0B0
:1023B000FC96DF01ECE3F0E00E94D1130895EC936A
:1023C000EB81F0E0FD96DF01ECE3F0E00E94D11339
:1023D0000895EC93EA81F0E008957C96DF01ECE348
:1023E000F0E00E94D1130895EA81F0E008957D960F
:1023F000DF01ECE3F0E00E94D11308957E96DF0147
:10240000ECE3F0E00E94D11308957F96DF01ECE346
:10241000F0E00E94D1130895B096DF01ECE3F0E004
:102420000E94D1130895AA5AB94FC7CEE053F94F6D
:10243000E081EC935CCEAC56B94FBFCEE45FF84F71
:10244000E081EC930895F0E0E85BF84F0895A6E092
:10245000B0E00E94B113E05AFD4FDF01EE27A10F5B
:10246000BE1FEC910895E981F0E00895A0E0A083FB
:10247000FACFAFEFA083F7CFE22FF0E00895A3E00B
:10248000B0E00E94ED13E1300895E1E0EA930E948C
:10249000BA027E2E0895E2E0EA930E94BA024E2E1E
:1024A0000895A5E0B0E00E94ED130895DF01F0016A
:1024B000E456FD4FE081EC9380CE0E94C0080C945E
:1024C00032080E94C0080C947908BF01A4E0B0E073
:1024D0000E94ED13F0E0DF01EAE0F0E00895F0E0A3
:1024E000DF01EAE0F0E00895A4E0B0E00E94ED131F
:1024F0000895EAE4F3E0FA93EA930895E1E0EA93B9
:102500000E9470040E94EA03F4CFE2E0EA930E9482
:1025100070040C94EA03E1E0EA930C9470040E94C6
:10252000EA03EAE3F4E0FA93EA9308950E94EA03E7
:102530003ECEFA93EA93EFCFFA93EA93E4E0EA937C
:102540000895EAE2F5E0FA93EA930895E2EAF5E005
:10255000FA93EA93E1E0EA930895FA93EA93E1E0CB
:10256000EA930895FA93EA93E2E0EA930895AD813D
:10257000BE81AE0FBF1FEC910895E450F84F0F01DC
:10258000E081EE0FAE2FFB01E054F84FE081F0E068
:10259000E078F0700E94A5130E94A313EA2BD001EB
:1025A000EC930895E054F84F0F01BECDAE2FFB0120
:1025B000E450F84FE081E170E795E0E0E795EA2B21
:1025C000D001EC930895BF01E2E0E29FF00108958D
:1025D000E054F84F0F01E081EE0FAE2FFB0108959C
:1025E000E081E170E795E0E0E795EA2BD001EC931C
:1025F00004CEEC91F0E0F595E795EC930895A09169
:102600003B08B0E0AC56B94FE0913B08F0E00895CC
:10261000E081EC93E0913B08F0E00F010895F5971D
:10262000EC56F94FDF01F001BE970895E0913B08A9
:10263000EF5FE0933B080895F497EC56F94FDF0104
:10264000F001BC9708950E94F913A3E0B0E0E0E028
:102650000E94F9130895E0E00E94F9130C94EA0334
:10266000E0913B08F0E0F797BF01EC56F94F0F01FE
:102670000895E0913B08F0E0BF010895FB01F69753
:10268000AE0FBF1FEC91D001EC9308950E94F91397
:102690000C94EA03F497EC56F94FDF01F001BA9776
:1026A0000895E0913E08F0E00895E054F84FAFEF50
:1026B000A083F7CFE0913E08EF5FE0933E080895D6
:1026C000EE0FFF1FE65EF94FE081EC93EACFEE0FCD
:1026D000FF1FE55EF94FE081EC930895E0913F081C
:1026E000F0E0BF010895A1E0B0E00E94ED13E030FA
:1026F0000895F0E0E45FF84FA0E0A0830895E2E0E1
:10270000EA9324CFE3E0EA93EAE3F4E02BCFEA9301
:10271000EAE3F4E022CFE991F991309639F080EDC7
:1027200097E00197F1F7A8953197C9F70895F195CA
:10273000E195F0400895EE230E2EEA2F19F0EE0FEA
:102740000A94E9F70895F595E795F595E795F595D8
:10275000E795F595E7950895EA17E1E009F0EE278A
:102760000895FA9FF02DEB9FF00DEA9FE02DF10DFB
:1027700008950024112490E1AA0FBB1F001C111C16
:102780000E1A1F0A18F40E0E1F1E01C0A1609A95A2
:1027900099F7FD01D001089512D0EBDF0EF4C7DFE9
:1027A0000895E894B7FF04C0A095B0951196689479
:1027B000F7FDBDDFDEDFFD010EF4B9DF0895E8941B
:1027C000F7FF02C0B4DF6894B7FF06C0A095B095CC
:1027D000119600F8039400FA0895E199FECFFF9353
:1027E000FFB7F894AEBBBFBBE09AEDB3FFBFFF915C
:1027F0000895E19B02C0A895FCCF9FB7F894AEBBAB
:10280000BFBBE09A8DB3E81719F0EDBBE29AE19AED
:102810009FBF08955A934A933A932A931A930A931F
:1028200008955D814C813B812A8119810881089539
:00000001FF
